:100000000C94DF000C94B90C0C94E00C0C940701D8
:100010000C9407010C9407010C9407010C94070140
:100020000C9407010C9407010C9407010C94070130
:100030000C9407010C9407010C9407010C94070120
:100040000C94070D0C9407010C9407010C94070104
:100050000C9407010C9407010C9407010C94070100
:100060000C9407010C940701000000080002010035
:100070000003040700000000000000000102040863
:100080001020408001020408102001020408102002
:10009000040404040404040402020202020203032E
:1000A00003030303000000002300260029000000D2
:1000B0000000250028002B0000000000240027007D
:1000C0002A0000407A10F35A00A0724E180900105E
:1000D000A5D4E80000E87648170000E40B540200BD
:1000E00000CA9A3B000000E1F505000080969800E8
:1000F000000040420F000000A08601000000102711
:1001000000000000E80300000000640000000000A0
:100110000A00000000000100000000002C76D888D2
:10012000DC674F0823DFC1DFAE59E1B1B796E5E3E5
:10013000E453C63AE651997696E8E6C28426EB89FE
:100140008C9B62ED407C6FFCEFBC9C9F40F2BAA59B
:100150006FA5F490055A2AF75C936B6CF9676DC133
:100160001BFCE0E40D47FEF520E6B500D0ED902E37
:100170000300943577050080841E080000204E0A95
:10018000000000C80C333333330F986E12831141D3
:10019000EF8D2114893BE65516CFFEE6DB18D1849E
:1001A0004B381BF77C1D901DA4BBE42420328472C5
:1001B0005E228100C9F124ECA1E53D27F90A112452
:1001C0001FBECFEFD8E0DEBFCDBF11E0A0E0B1E0B1
:1001D000E8E7F8E202C005900D92A43AB107D9F71A
:1001E00022E0A4EAB1E001C01D92A431B207E1F718
:1001F00011E0CEEBD1E004C02297FE010E949A11DB
:10020000CC3BD107C9F70E94AA0F0C943A140C9466
:1002100000000F931F93CF93DF9300D000D0CDB792
:10022000DEB78091BE01882309F493C0809100015C
:10023000909101010E948C0E892B61F0809109013F
:1002400090E00A9724F4809109018F5F0CC010920E
:1002500009010BC080910901882321F080910901D7
:10026000815001C08AE080930901E091090184E096
:10027000E89FF0011124E65FFE4F80819181A28109
:10028000B3818093CF019093D001A093D101B0931B
:10029000D20184EA91E00E94A10B65E671E084EA54
:1002A00091E00E94F30E40E065E084EA91E00E9454
:1002B000A80B809109018630C8F44091CF0150917C
:1002C000D0016091D1017091D2012AE030E084EA3E
:1002D00091E00E944B0F80910901882309F48DC0A1
:1002E00080910901813009F0B9C087C06091CF01C8
:1002F0007091D0018091D1019091D201209105019E
:1003000030910601409107015091080129833A83F9
:100310004B835C830E94541029813A814B815C811C
:100320000E94BE0F0E9426106093CE016091CE0104
:100330004AE050E084EA91E00E94A20F8091090116
:10034000863009F4A0C080910901873009F062C0AD
:100350009AC080910001909101010E948C0E892B1E
:1003600031F140913A0150913B0160913C01709113
:100370003D0180913E0190913F01A0914001B091DB
:1003800041010091CF011091D0012091D101309114
:10039000D201800F911FA21FB31F481759076A0788
:1003A0007B070CF474C081E08093BD0170C0809124
:1003B0003E0190913F01A0914001B0914101009117
:1003C000CF011091D0012091D1013091D201409103
:1003D0003601509137016091380170913901801BCD
:1003E000910BA20BB30B84179507A607B7070CF464
:1003F0004EC081E08093BC014AC086E08093CD016D
:100400006091CD0140E084EA91E00E94A80B6BE688
:1004100071E018C0809109018830B9F1809109011B
:10042000893099F1809109018A3019F488E080932C
:10043000CD016091CD0140E084EA91E00E94A80BDB
:100440006FE671E084EA91E00F900F900F900F90AB
:10045000DF91CF911F910F910C94F30E80910901C0
:10046000823041F080910901833021F080910901AF
:10047000843011F487E0C2CF80910901853009F002
:10048000BFCF88E0BBCF86E0D2CF87E0D0CF0F9040
:100490000F900F900F90DF91CF911F910F910895C2
:1004A0000C94CE110C94D61168EE73E080E090E0CD
:1004B0000E94740D20E042E060E184EA91E00E9435
:1004C000C20B84EA91E00E94A10B40E060E084EA64
:1004D00091E00C94A80B8091040160E00E941D0E35
:1004E0008091040161E00C94560E0F931F93CF93FB
:1004F000DF9300D000D0CDB7DEB784EA91E00E9450
:10050000A10B63E771E084EA91E00E94F30E40E002
:100510006DE084EA91E00E94A80B6FE671E084EA46
:1005200091E00E94F30E40E065E084EA91E00E94D1
:10053000A80B6091D3017091D4018091D501909165
:10054000D6010FEB11E023E044E00E94AD11B801A9
:1005500084EA91E00E94F30E41E060E084EA91E0D9
:100560000E94A80B65E671E084EA91E00E94F30E18
:1005700041E065E084EA91E00E94A80B80910901C6
:100580008630C0F44091CF015091D0016091D101EB
:100590007091D2012AE030E084EA91E00E944B0F92
:1005A000809109018823C1F180910901813009F00E
:1005B00072C032C06091CF017091D0018091D101A1
:1005C0009091D201209105013091060140910701DF
:1005D0005091080129833A834B835C830E94541015
:1005E00029813A814B815C810E94BE0F0E942610B6
:1005F0006093CE016091CE014AE050E084EA91E040
:100600000E94A20F80910901863009F459C080919F
:100610000901873071F454C086E08093CD01609168
:10062000CD0141E084EA91E00E94A80B6BE671E005
:100630001AC080910901883009F444C080910901F1
:10064000893009F43FC0809109018A3019F488E0AB
:100650008093CD016091CD0141E084EA91E00E9458
:10066000A80B6FE671E084EA91E00E94F30E41E08E
:100670006DE084EA91E00E94A80B69E771E084EAEA
:1006800091E00F900F900F900F90DF91CF911F91FD
:100690000F910C94F30E80910901823079F08091D2
:1006A0000901833059F080910901843039F080913B
:1006B0000901853009F0B3CF88E0AFCF87E0ADCF37
:1006C00086E0C6CF87E0C4CFCF92DF92EF92FF9251
:1006D000CF93DF93EC016A017B01642F0E945202E9
:1006E0009927F7FC9A958F2D7E2D6D2DCE010196C1
:1006F0000E945202B701992777FD9095892FCE016C
:1007000002960E9452026F2D772788279927CE01E3
:100710000396DF91CF91FF90EF90DF90CF900C94F4
:100720005202CF92DF92EF92FF920F931F93CF93DB
:100730006B017C01CB010E945002182FC60101966B
:100740000E945002C82FC60102960E945002082F34
:10075000C60103960E945002C82E8C2F90E0A0E0A4
:10076000B0E06627782F892F9A2F610F711D811DA8
:10077000911D10E020E030E0980111270027600F64
:10078000711F821F931FD12CE12CF12CFC2CEE2425
:10079000DD24CC246C0D7D1D8E1D9F1DCF911F91DE
:1007A0000F91FF90EF90DF90CF900895CF92DF925E
:1007B000EF92FF92CF93DF936B017C0160E0809119
:1007C0005F010E94560E60E0809160010E94560E0B
:1007D000CFE1D0E0D701C6010C2E04C0B695A79595
:1007E000979587950A94D2F780FF02C061E001C017
:1007F00060E080915E010E94560E61E080915F0191
:100800000E94560E60E080915F010E94560E219773
:1008100008F761E080916001DF91CF91FF90EF9048
:10082000DF90CF900C94560E4F925F926F927F9212
:100830008F929F92AF92BF92CF92DF92EF92FF92F0
:10084000CF93DF9300D000D0CDB7DEB780E893E23E
:10085000A3E4B0E08093F3019093F401A093F50139
:10086000B093F60180EC91E9A1E2B0E08093EF0152
:100870009093F001A093F101B093F20180913E01B9
:1008800090913F01A0914001B0914101803C91497C
:10089000A142B10570F080913E0190913F01A0917D
:1008A0004001B091410181389342A344B10508F45D
:1008B000CCC280EC91E9A1E2B0E08093F301909387
:1008C000F401A093F501B093F60180EE98ECA0E15D
:1008D000B0E08093EF019093F001A093F101B09309
:1008E000F20180913E0190913F01A0914001B091B1
:1008F0004101803E984CA041B10570F080913E01CD
:1009000090913F01A0914001B0914101803C9149FB
:10091000A142B10508F4AEC280EE98ECA0E1B0E0CF
:100920008093F3019093F401A093F501B093F60145
:1009300080E794E6A8E0B0E08093EF019093F001A7
:10094000A093F101B093F20180913E0190913F019B
:10095000A0914001B091410180379446A840B10573
:1009600070F080913E0190913F01A0914001B091C3
:100970004101803E984CA041B10508F494C280E743
:1009800094E6A8E0B0E08093F3019093F401A09383
:10099000F501B093F60188E392E3A4E0B0E0809320
:1009A000EF019093F001A093F101B093F2018091D7
:1009B0003E0190913F01A0914001B09141018833E7
:1009C0009243A440B10570F080913E0190913F01A7
:1009D000A0914001B091410180379446A840B105F3
:1009E00008F47AC288E392E3A4E0B0E08093F301D4
:1009F0009093F401A093F501B093F6018CE199E195
:100A0000A2E0B0E08093EF019093F001A093F10198
:100A1000B093F20180913E0190913F01A09140017D
:100A2000B09141018C319941A240B10570F08091A3
:100A30003E0190913F01A0914001B0914101883366
:100A40009243A440B10508F460C28CE199E1A2E0B0
:100A5000B0E08093F3019093F401A093F501B0937B
:100A6000F6018EE89CE0A1E0B0E08093EF01909366
:100A7000F001A093F101B093F20180913E019091B9
:100A80003F01A0914001B09141018E389C40A140AE
:100A9000B10570F080913E0190913F01A09140011D
:100AA000B09141018C319941A240B10508F446C290
:100AB0008EE89CE0A1E0B0E08093F3019093F40114
:100AC000A093F501B093F60187E496E8A0E0B0E0CA
:100AD0008093EF019093F001A093F101B093F201A4
:100AE00080913E0190913F01A0914001B091410160
:100AF00087349648A105B10570F080913E01909130
:100B00003F01A0914001B09141018E389C40A1402D
:100B1000B10508F42CC220913E0130913F01409173
:100B20004001509141018090FF0190900002A090FF
:100B30000102B0900202C501B4010E945B1161384C
:100B40007E4E8643910568F081E090E0A0E0B0E041
:100B50008093F7019093F801A093F901B093FA0103
:100B600008C01092F7011092F8011092F90110924A
:100B7000FA0120913E0130913F0140914001509196
:100B80004101C0905601D0905701E0905801F0907B
:100B90005901C501B4010E945B11A70196010E9491
:100BA0006B11CA01B9010E9452100E948F100E945D
:100BB00026102B013C01609307027093080280937A
:100BC000090290930A0220913E0130913F01409129
:100BD00040015091410180915A0190915B01A09197
:100BE0005C01B0915D0189839A83AB83BC83C501AD
:100BF000B4010E945B114B015C01A3019201C7018A
:100C0000B6010E945B11861A970AA80AB90AA501C3
:100C1000940169817A818B819C810E945B11A7017B
:100C200096010E946B1120930302309304024093BB
:100C3000050250930602DA01C90163E0880F991F8B
:100C4000AA1FBB1F6A95D1F7B301A201EFE0440FC1
:100C5000551F661F771FEA95D1F7842B952BA62B7E
:100C6000B72B8093EB019093EC01A093ED01B0932F
:100C7000EE018091F7019091F801A091F901B091F6
:100C8000FA01FBE1880F991FAA1FBB1FFA95D1F744
:100C9000409152015091530160915401709155015E
:100CA0002FE0440F551F661F771F2A95D1F7842B1D
:100CB000952BA62BB72B816049805A806B807C8056
:100CC00033E0440C551C661C771C3A95D1F78429F7
:100CD0009529A629B7298093E7019093E801A0936D
:100CE000E901B093EA0180914E0190914F01A091EA
:100CF0005001B091510147E1880F991FAA1FBB1FF6
:100D00004A95D1F74091FB015091FC016091FD01A2
:100D10007091FE01E4E1440F551F661F771FEA95AD
:100D2000D1F7842B952BA62BB72B846040914A01D9
:100D300050914B0160914C0170914D01FCE0440FCA
:100D4000551F661F771FFA95D1F7842B952BA62B7D
:100D5000B72B409146015091470160914801709135
:100D6000490125E0440F551F661F771F2A95D1F7CB
:100D7000842B952BA62BB72B409142015091430118
:100D8000609144017091450133E0440F551F661F87
:100D9000771F3A95D1F7842B952BA62BB72B8093F1
:100DA000DB019093DC01A093DD01B093DE01609143
:100DB000D7017091D8018091D9019091DA010E94F8
:100DC000D6036091DB017091DC018091DD0190918F
:100DD000DE010E94D6036091DF017091E0018091F5
:100DE000E1019091E2010E94D6036091E3017091CC
:100DF000E4018091E5019091E6010E94D6036091A3
:100E0000E7017091E8018091E9019091EA010E9467
:100E1000D6036091EB017091EC018091ED0190910E
:100E2000EE010F900F900F900F90DF91CF91FF90F8
:100E3000EF90DF90CF90BF90AF909F908F907F907A
:100E40006F905F904F900C94D6031092FB0110921C
:100E5000FC011092FD011092FE0181E090E0A0E003
:100E6000B0E08093FF0190930002A0930102B09341
:100E700002021FCD81E090E0A0E0B0E08093FB0192
:100E80009093FC01A093FD01B093FE0182E090E0FD
:100E9000A0E0B0E08093FF0190930002A0930102D4
:100EA000B093020239CD82E090E0A0E0B0E0809300
:100EB000FB019093FC01A093FD01B093FE0184E03F
:100EC00090E0A0E0B0E08093FF0190930002A09337
:100ED0000102B093020253CD83E090E0A0E0B0E0C5
:100EE0008093FB019093FC01A093FD01B093FE0160
:100EF00088E090E0A0E0B0E08093FF0190930002D2
:100F0000A0930102B09302026DCD84E090E0A0E0D6
:100F1000B0E08093FB019093FC01A093FD01B0939E
:100F2000FE0180E190E0A0E0B0E08093FF019093AB
:100F30000002A0930102B093020287CD85E090E009
:100F4000A0E0B0E08093FB019093FC01A093FD0131
:100F5000B093FE0180E290E0A0E0B0E08093FF015A
:100F600090930002A0930102B0930202A1CD86E00B
:100F700090E0A0E0B0E08093FB019093FC01A0938F
:100F8000FD01B093FE0180E490E0A0E0B0E080932A
:100F9000FF0190930002A0930102B0930202BBCD27
:100FA000CF93DF9300D000D0CDB7DEB761E0809162
:100FB00060010E941D0E61E0809160010E94560E4A
:100FC00061E080915F010E941D0E60E080915F01F1
:100FD0000E94560E61E080915E010E941D0E60E04D
:100FE00080915E010E94560E82E49EE4A6E0B8E184
:100FF0008093E3019093E401A093E501B093E601AF
:1010000083EB94E0A0E0B0E08093DF019093E001F7
:10101000A093E101B093E2018CE390E8A0ECB0E092
:101020008093DB019093DC01A093DD01B093DE019E
:1010300085E090E0A8E5B0E08093D7019093D801D7
:10104000A093D901B093DA010E941404EE24E39432
:1010500046E0D42E57E0C52E68E0F62E80910401BC
:101060000E948C0E892B41F08091BD01811104C03A
:101070008091BC01882391F380E00E94A70C8091AD
:1010800004010E948C0E892B09F0F4C0E092BE018D
:10109000809104010E948C0E892BA1F48091C901DA
:1010A0009091CA01A091CB01B091CC010196A11DF4
:1010B000B11D8093C9019093CA01A093CB01B09355
:1010C000CC01E6CF8091C9019091CA01A091CB01DA
:1010D000B091CC01813A9648A140B1051CF14091F4
:1010E0003E0150913F01609140017091410180E0CB
:1010F00090E00E9464036091090185E090E00E9405
:10110000520284EA91E00E94A10B6CE771E084EA4C
:1011100091E00E94F30E68EE73E080E090E00E94A0
:10112000740D98C08CB3813009F48CBB42E050E060
:1011300069E071E080E00E94870C84EA91E00E94FF
:10114000A10B65E671E084EA91E00E94F30E40E0B5
:1011500065E084EA91E00E94A80B80910901863045
:10116000C0F44091CF015091D0016091D1017091B4
:10117000D2012AE030E084EA91E00E944B0F809196
:101180000901882309F42BC1809109018130A1F55F
:1011900026C16091CF017091D0018091D1019091D1
:1011A000D201209105013091060140910701509133
:1011B000080129833A834B835C830E945410298160
:1011C0003A814B815C810E94BE0F0E942610609381
:1011D000CE016091CE014AE050E084EA91E00E94A5
:1011E000A20F80910901863009F4FFC080910901A6
:1011F000873009F006C1F9C080910901823009F4F5
:10120000F1C080910901833009F4ECC0809109019B
:10121000843009F4E7C080910901853011F4F0921F
:10122000CD016091CD0140E084EA91E00E94A80BDD
:101230006BE671E084EA91E00E94F30E8091040174
:101240000E948C0E892BD1F7809104010E948C0E94
:10125000892BD1F380E00E94A70C1092BE0110925E
:10126000C9011092CA011092CB011092CC010E94C8
:101270007502A9C08091BD018823A9F04091CF01DA
:101280005091D0016091D1017091D20180913E01C5
:1012900090913F01A0914001B0914101840F951FB1
:1012A000A61FB71F18C08091BC018823E1F04091B0
:1012B000CF015091D0016091D1017091D201809104
:1012C0003E0190913F01A0914001B0914101841BEA
:1012D000950BA60BB70B80933E0190933F01A09313
:1012E0004001B09341011092BD011092BC010E94D7
:1012F000140460913E0170913F01809140019091F2
:101300004101209105013091060140910701509162
:10131000080129833A834B835C830E9454102981FE
:101320003A814B815C810E94BE0F6093D301709320
:10133000D4018093D5019093D6016091D30170912F
:10134000D4018091D5019091D60120E030E048ECA5
:1013500052E40E94571118160CF065C06091D30139
:101360007091D4018091D5019091D60120E030E0B8
:101370004AE754E40E94BA0F87FF55C040E06CE092
:1013800084EA91E00E94A80B6DE871E084EA91E0A4
:101390000E94F30E6091D3017091D4018091D50128
:1013A0009091D6010FEB11E023E044E00E94AD11D3
:1013B00040E065E084EA91E00E94A80BB80184EA6D
:1013C00091E00E94F30E8CB3813009F48CBB42E0B3
:1013D00050E069E071E080E00E94870C3FCED0923F
:1013E000CD011FCFC092CD011CCFD092CD01609115
:1013F000CD0140E084EA91E00E94A80B6FE671E025
:1014000019CF80910901883059F080910901893004
:1014100039F0809109018A3051F7F092CD01E7CF80
:10142000C092CD01E4CF6091D3017091D40180913D
:10143000D5019091D60120E030E048EC52E40E94C2
:10144000BA0F87FFA7CF40E06BE084EA91E00E94EB
:10145000A80B6CE871E09ACF84EA91E00E94A10B9E
:101460006FE871E084EA91E00C94F30ECF93DF9380
:1014700000D000D0CDB7DEB760E070E0CB010E94B5
:10148000910360933E0170933F01809340019093DC
:10149000410185E090E00E94500280930901409153
:1014A0003601509137016091380170913901809176
:1014B0003E0190913F01A0914001B09141018417FC
:1014C0009507A607B7070CF485C040913E015091DF
:1014D0003F01609140017091410180913A019091EA
:1014E0003B01A0913C01B0913D0184179507A607EF
:1014F000B7070CF46FC080910901809109018B300E
:1015000008F068C0E091090184E0E89FF00111242F
:10151000E65FFE4F80819181A281B3818093CF01EC
:101520009093D001A093D101B093D20160913E017C
:1015300070913F01809140019091410120910501FE
:1015400030910601409107015091080129833A83A7
:101550004B835C830E94541029813A814B815C81CA
:101560000E94BE0F6093D3017093D4018093D50184
:101570009093D6010E946B020E9454020E942C0A92
:1015800068EE73E080E090E00E94740D0E947502A6
:1015900042E050E069E071E080E00E94870C8091B9
:1015A00002019091030160E00E941D0E80910201F2
:1015B0009091030161E00E94560E8091000190918C
:1015C000010162E00F900F900F900F90DF91CF918B
:1015D0000C941D0E8EED9BE8A4E0B0E080933E01DC
:1015E00090933F01A0934001B093410110920901F3
:1015F00089CFCF92EF920F9379E0C72EE8E0EE2EDD
:1016000007E026E045E064E084EA91E00E94600C97
:101610000F91EF90CF900895CF93DF93EC0160E0AE
:101620008E810E94560E81E090E00E94AE0D61E036
:101630008E810E94560E81E090E00E94AE0D60E027
:101640008E810E94560E84E690E0DF91CF910C943B
:10165000AE0DEF92FF920F931F93CF93DF938C0108
:10166000C0E0D0E0E62EF12CB7010C2E02C075953B
:1016700067950A94E2F76170F801EC0FFD1F87810E
:101680000E94560E2196C430D10571F7C801DF9132
:10169000CF911F910F91FF90EF900C940C0BEF9254
:1016A000FF920F931F93CF93DF938C01C0E0D0E0A4
:1016B000E62EF12CB7010C2E02C0759567950A94A1
:1016C000E2F76170F801EC0FFD1F87810E94560E52
:1016D0002196C830D10571F7C801DF91CF911F91D4
:1016E0000F91FF90EF900C940C0B1F93CF93DF930F
:1016F000EC01162F642F8C810E94560E8D818F3F36
:1017000019F060E00E94560E8F85612F84FF06C09D
:10171000CE01DF91CF911F910C944F0B70E084E0CC
:10172000759567958A95E1F7CE010E94290B612F87
:10173000CE01DF91CF911F910C94290B40E00C94C6
:10174000750B61E00E949E0B80ED97E00C94AE0D4E
:10175000443008F043E0FC012389421710F04FEFBA
:10176000420FFC01E40FF11D2489260F2068622F2F
:101770000C949E0BFC016089262F2460208B6C60EA
:101780000C949E0B0F931F93CF93DF93EC01423089
:1017900018F08F8588608F874B8B1C8A80E48D8B37
:1017A0006E8B70E0605C7F4F6F8B222329F041309D
:1017B00019F48F8584608F8761E08C810E941D0EF3
:1017C0008D818F3F19F061E00E941D0E61E08E81D6
:1017D0000E941D0E00E010E08F8584FF03C088E0AA
:1017E00090E002C084E090E00817190754F4FE016D
:1017F000E00FF11F61E087810E941D0E0F5F1F4FF8
:10180000EBCF80E593EC0E94AE0D60E08C810E94EE
:10181000560E60E08E810E94560E8D818F3F19F02A
:1018200060E00E94560E6F8564FD1DC063E0CE012E
:101830000E94290B84E991E10E94AE0D63E0CE0184
:101840000E94290B84E991E10E94AE0D63E0CE0174
:101850000E94290B86E990E00E94AE0D62E0CE0165
:101860000E94290B16C06062CE010E949E0B84E983
:1018700091E10E94AE0D6F856062CE010E949E0BC9
:1018800086E990E00E94AE0D6F856062CE010E94F5
:101890009E0B6F856062CE010E949E0B84E0888B58
:1018A000CE010E94BA0BCE010E94A10B82E0898B6F
:1018B00066E0CE01DF91CF911F910F910C949E0BAA
:1018C000CF92EF920F93FC01138212828FE991E085
:1018D0009183808364838FEF85834683278300878A
:1018E000E186C2861386148615861686178620E042
:1018F00041E060E1CF010F91EF90CF900C94C20BCB
:1019000041E00E94750B81E090E0089508958230D7
:10191000E8F4E82FF0E0EE0FFF1FEF59FE4F718360
:101920006083813041F0809169008C7F842B8093AB
:101930006900E89A089580916900440F551F440F8B
:10194000551F837F842B80936900E99A0895823024
:1019500078F4813011F0E89801C0E998E82FF0E0C0
:10196000EE0FFF1FEF59FE4F86E89CE091838083C6
:1019700008951F920F920FB60F9211242F933F9349
:101980004F935F936F937F938F939F93AF93BF9387
:10199000EF93FF93E0916101F09162010995FF914E
:1019A000EF91BF91AF919F918F917F916F915F91D7
:1019B0004F913F912F910F900FBE0F901F90189550
:1019C0001F920F920FB60F9211242F933F934F93B4
:1019D0005F936F937F938F939F93AF93BF93EF9397
:1019E000FF93E0916301F09164010995FF91EF91FC
:1019F000BF91AF919F918F917F916F915F914F9127
:101A00003F912F910F900FBE0F901F9018951F922E
:101A10000F920FB60F9211242F933F938F939F93A2
:101A2000AF93BF9380910C0290910D02A0910E0292
:101A3000B0910F0230910B0223E0230F2D3720F4D9
:101A40000196A11DB11D05C026E8230F0296A11D18
:101A5000B11D20930B0280930C0290930D02A09372
:101A60000E02B0930F028091100290911102A0918A
:101A70001202B09113020196A11DB11D80931002B4
:101A800090931102A0931202B0931302BF91AF91F1
:101A90009F918F913F912F910F900FBE0F901F90AC
:101AA00018953FB7F8948091100290911102A0917F
:101AB0001202B091130226B5A89B05C02F3F19F062
:101AC0000196A11DB11D3FBF6627782F892F9A2F40
:101AD000620F711D811D911D42E0660F771F881FE7
:101AE000991F4A95D1F708958F929F92AF92BF9216
:101AF000CF92DF92EF92FF926B017C010E94510D19
:101B00004B015C01C114D104E104F104F1F00E9425
:101B1000B90F0E94510D681979098A099B09683E1D
:101B200073408105910570F321E0C21AD108E108E4
:101B3000F10888EE880E83E0981EA11CB11CC11428
:101B4000D104E104F10429F7DDCFFF90EF90DF909D
:101B5000CF90BF90AF909F908F9008958230910565
:101B600038F0880F991F880F991F05970197F1F793
:101B70000895789484B5826084BD84B5816084BD05
:101B800085B5826085BD85B5816085BDEEE6F0E0F6
:101B9000808181608083E1E8F0E010828081826052
:101BA0008083808181608083E0E8F0E080818160D3
:101BB0008083E1EBF0E0808184608083E0EBF0E003
:101BC000808181608083EAE7F0E0808184608083A7
:101BD0008081826080838081816080838081806851
:101BE00080831092C1000895833081F028F4813001
:101BF00099F08230A1F008958730A9F08830B9F0CB
:101C00008430D1F4809180008F7D03C0809180006A
:101C10008F7780938000089584B58F7702C084B554
:101C20008F7D84BD08958091B0008F7703C080912F
:101C3000B0008F7D8093B0000895CF93DF9390E044
:101C4000FC01E458FF4F2491FC01E057FF4F8491C1
:101C5000882349F190E0880F991FFC01E854FF4F59
:101C6000A591B49182559F4FFC01C591D4919FB726
:101C7000611108C0F8948C91209582238C938881FF
:101C800082230AC0623051F4F8948C91322F30953F
:101C900083238C938881822B888304C0F8948C9151
:101CA000822B8C939FBFDF91CF9108950F931F9349
:101CB000CF93DF931F92CDB7DEB7282F30E0F90125
:101CC000E859FF4F8491F901E458FF4F1491F9014D
:101CD000E057FF4F04910023C9F0882321F0698366
:101CE0000E94F40D6981E02FF0E0EE0FFF1FE25536
:101CF000FF4FA591B4919FB7F8948C91611103C0E7
:101D00001095812301C0812B8C939FBF0F90DF9191
:101D1000CF911F910F910895CF93DF93282F30E03B
:101D2000F901E859FF4F8491F901E458FF4FD4912C
:101D3000F901E057FF4FC491CC2391F081110E942B
:101D4000F40DEC2FF0E0EE0FFF1FEC55FF4FA591C7
:101D5000B4912C912D2381E090E021F480E002C029
:101D600080E090E0DF91CF910895CF92DF92EF92E3
:101D7000FF920F931F93CF93DF937C016A01EB01D6
:101D800000E010E00C151D0571F06991D701ED918F
:101D9000FC910190F081E02DC7010995892B19F084
:101DA0000F5F1F4FEFCFC801DF91CF911F910F91B0
:101DB000FF90EF90DF90CF9008956115710581F04D
:101DC000DB010D900020E9F7AD0141505109461BA0
:101DD000570BDC01ED91FC910280F381E02D099419
:101DE00080E090E008950C94DD0EDC01ED91FC9113
:101DF0000190F081E02D09948F929F92AF92BF9253
:101E0000DF92EF92FF920F931F93CF93DF93CDB7A3
:101E1000DEB7A1970FB6F894DEBF0FBECDBF7C0131
:101E2000F42FD52ECB0119A2223008F42AE08E011E
:101E30000F5D1F4F822E912CA12CB12C6F2F7D2D69
:101E4000A50194010E946B11F22FD32ECA010150FB
:101E500011096A3014F4E0E301C0E7E3E60FD801AA
:101E6000EC93232B242B252B49F7B801C7010E94A3
:101E7000DD0EA1960FB6F894DEBF0FBECDBFDF9189
:101E8000CF911F910F91FF90EF90DF90BF90AF9097
:101E90009F908F900895CF92DF92EF92FF920F93D1
:101EA0001F93CF93DF93EC016A017B01211531056C
:101EB00079F4E881F9810190F081E02D642FDF91C0
:101EC000CF911F910F91FF90EF90DF90CF900994E9
:101ED0002A303105E9F477FF1AC06DE20E94F50E51
:101EE0008C0144275527BA014C195D096E097F09F9
:101EF0002AE0CE010E94FC0E800F911FDF91CF914E
:101F00001F910F91FF90EF90DF90CF9008952AE0FE
:101F1000B701A601CE01DF91CF911F910F91FF90E4
:101F2000EF90DF90CF900C94FC0E2115310541F419
:101F3000DC01ED91FC910190F081E02D642F09947A
:101F40000C94FC0E9A01462F50E060E070E00C9477
:101F5000950F08950E94B90D0E94A90F0E94360A9C
:101F6000C0E0D0E00E94D0072097E1F30E9400007B
:101F7000F9CF0895E7D008F481E008950CD046C168
:101F80003ED140F035D130F021F45F3F19F0FEC072
:101F9000511187C12AC14BD198F39923C9F3552315
:101FA000B1F3951B550BBB27AA276217730784074C
:101FB00038F09F5F5F4F220F331F441FAA1FA9F302
:101FC00033D00E2E3AF0E0E830D091505040E695F4
:101FD000001CCAF729D0FE2F27D0660F771F881F55
:101FE000BB1F261737074807AB07B0E809F0BB0B44
:101FF000802DBF01FF2793585F4F2AF09E3F510568
:1020000068F0C4C04EC15F3FECF3983EDCF38695A8
:1020100077956795B795F7959F5FC9F7880F911DDD
:102020009695879597F90895E1E0660F771F881FC9
:10203000BB1F621773078407BA0720F0621B730B7C
:10204000840BBA0BEE1F88F7E0950895F8D088F05E
:102050009F5790F0B92F9927B751A0F0D1F0660F94
:10206000771F881F991F1AF0BA95C9F712C0B130AF
:1020700081F016D1B1E0089513C1672F782F88271A
:10208000B85F39F0B93FCCF3869577956795B395EE
:10209000D9F73EF490958095709561957F4F8F4F5D
:1020A0009F4F0895E89409C097FB3EF49095809562
:1020B000709561957F4F8F4F9F4F9923A9F0F92F0E
:1020C00096E9BB279395F695879577956795B7958C
:1020D000F111F8CFFAF4BB0F11F460FF1BC06F5F72
:1020E0007F4F8F4F9F4F16C0882311F096E911C084
:1020F000772321F09EE8872F762F05C0662371F0A5
:1021000096E8862F70E060E02AF09A95660F771FB8
:10211000881FDAF7880F9695879597F90895A9D0C3
:1021200080F09F3740F491110EF0BBC060E070E08A
:1021300080E89FEB089526F41B16611D711D811D1B
:102140002BC045C0990F0008550FAA0BE0E8FEEF21
:1021500016161706E807F907C0F012161306E4076B
:10216000F50798F0621B730B840B950B39F40A2664
:1021700061F0232B242B252B21F408950A2609F442
:10218000A140A6958FEF811D811D089597F99F6746
:1021900080E870E060E00895882371F4772321F0EF
:1021A0009850872B762F07C0662311F499270DC00E
:1021B0009051862B70E060E02AF09A95660F771FA9
:1021C000881FDAF7880F9695879597F908959F3FAE
:1021D00031F0915020F4879577956795B795880FE2
:1021E000911D9695879597F908959FEF80EC089536
:1021F00000240A94161617061806090608950024E6
:102200000A9412161306140605060895092E03945F
:10221000000C11F4882352F0BB0F40F4BF2B11F4D3
:1022200060FF04C06F5F7F4F8F4F9F4F089557FD32
:102230009058440F551F59F05F3F71F04795880F34
:1022400097FB991F61F09F3F79F0879508951216CB
:1022500013061406551FF2CF4695F1DF08C0161677
:1022600017061806991FF1CF869571056105089428
:102270000895E5DFA0F0BEE7B91788F4BB279F38C3
:1022800060F41616B11D672F782F8827985FF7CF57
:10229000869577956795B11D93959639C8F30895FE
:1022A000E894BB2766277727CB0197F908954ADF83
:1022B00008F48FEF0895DB018F939F930E948D1197
:1022C000BF91AF91A29F800D911DA39F900DB29FD2
:1022D000900D11240895A1E21A2EAA1BBB1BFD012B
:1022E0000DC0AA1FBB1FEE1FFF1FA217B307E407F5
:1022F000F50720F0A21BB30BE40BF50B661F771F4D
:10230000881F991F1A9469F760957095809590952C
:102310009B01AC01BD01CF0108950E949E11A59FB4
:10232000900DB49F900DA49F800D911D11240895D0
:10233000EE0FFF1F0590F491E02D0994A29FB001CC
:10234000B39FC001A39F700D811D1124911DB29FE9
:10235000700D811D1124911D0895EF920F931F930D
:10236000CF93DF93E80147FF02C034E101C034E0BE
:10237000E42FFF27E7FDF095F7FF03C0F195E19506
:10238000F109E32E022F2E2FAE010E94E411CE019F
:10239000DF91CF911F910F91EF900895F999FECFA2
:1023A00092BD81BDF89A992780B50895262FF99995
:1023B000FECF1FBA92BD81BD20BD0FB6F894FA9A28
:1023C000F99A0FBE019608956F927F929F92AF92F5
:1023D000BF92CF92DF92EF92FF920F931F93CF9312
:1023E000DF93CDB7DEB729970FB6F894DEBF0FBEE7
:1023F000CDBF6A01B22E102F0C3320F4FF24F394CA
:10240000F00E02C04CE3F42E0F2D27E0AE014F5F1B
:102410005F4F0E9462137981272F2970213031F09C
:10242000E1FC06C0E0FC06C060E005C06DE203C050
:102430006BE201C060E2AE2DA07173FF36C066236F
:1024400011F084E001C083E08B1510F4B81A01C0CC
:10245000B12CA1110BC0F6018B2D90E2882319F04D
:1024600091938150FBCFCB0CD11CB12C662331F062
:10247000F601608396012F5F3F4F6901C601039605
:10248000E2FE05C02EE4F601208331E404C02EE60E
:10249000F601208331E631832283FC012B2D30E2CB
:1024A0002223F1F131932150FBCF72FF40C066230C
:1024B00011F084E001C083E08B1510F4B81A01C05C
:1024C000B12CA1110BC0F6018B2D90E2882319F0DD
:1024D00091938150FBCFCB0CD11CB12C662331F0F2
:1024E000F601608396012F5F3F4F6901C601039695
:1024F000E2FE07C029E4F60120832EE4218326E4CE
:1025000006C029E6F60120832EE6218326E62283F3
:10251000FC012B2D30E2222319F031932150FBCF07
:10252000FC01EB0DF11D10828EEF9FEFB7C0B1E003
:10253000611101C0B0E04B2F50E01816190624F4C9
:102540009C012F5F3F4F02C021E030E0240F351F78
:10255000112329F0412F50E04F5F5F4F02C040E050
:1025600050E0420F531F2B2D30E04217530714F455
:10257000B41A01C0B12C2E2D287159F4F6012B2D5F
:1025800030E2222319F031932150FBCFCB0CD11C28
:10259000B12CBB2331F0F601608396012F5F3F4FD2
:1025A0006901A1110BC0F6012B2D30E3222319F094
:1025B00031932150FBCFCB0CD11CB12CF80E0A81EA
:1025C000372F3071A32E74FF03C0013309F4FA943E
:1025D0001F142CF42F2D293018F028E001C021E021
:1025E000682F392F97FF02C060E030E0462F532F4D
:1025F000612C712C3EE2932EBC01621B71099B0180
:10260000DC01A41BB50BE1E0F0E0EC0FFD1FAE0F09
:10261000BF1FE12EF12CF194E194F1084F3FFFEF41
:102620005F0731F4F6019082B6016F5F7F4F6B0157
:10263000841795074CF02417350734F4BD01660D57
:10264000771DFB01118101C010E341505109FFEFDB
:102650006F1A7F0AB6016F5F7F4F4E155F0524F03A
:10266000F60110836B01DACF4817590739F40633A6
:1026700020F4053319F4A11001C011E3F601108311
:10268000FB018B2D90E2882319F091938150FBCFB1
:10269000FB01EB0DF11D108280E090E029960FB652
:1026A000F894DEBF0FBECDBFDF91CF911F910F9188
:1026B000FF90EF90DF90CF90BF90AF909F907F9072
:1026C0006F900895283008F027E03327DA01990F3A
:1026D000311D87FD916000966105710539F4326006
:1026E0002E5F3D9330E32A95E1F708959F3F30F048
:1026F00080387105610509F03C5F3C5F3D93913086
:1027000008F08068911DDF93CF931F930F93FF9282
:10271000EF92192F987F9695E92F96959695E90F48
:10272000FF27E45EFE4F99273327EE24FF24A701FD
:10273000E70105900894079428F4360FE71EF81E69
:10274000491F511D660F771F881F991F0694A1F717
:102750000590079428F4E70EF81E491F561FC11D67
:10276000770F881F991F661F0694A1F7059007949D
:1027700028F4F80E491F561FC71FD11D880F991F37
:10278000661F771F0694A1F70590079420F4490F60
:10279000561FC71FD81F990F661F771F881F0694E3
:1027A000A9F784911095177041F0D695C795579564
:1027B0004795F794E7941A95C1F7E2ECF0E0689436
:1027C0001590159135916591959105907FE27395DE
:1027D000E118F10A430B560BC90BD009C0F7E10C05
:1027E000F11E431F561FC91FD01D7EF4703311F414
:1027F0008A95E6CFE894015030F0080F0AF40027DC
:10280000021708F4202F2395022F7A3328F079E35A
:102810007D932A95E9F710C07D932A9589F6069451
:1028200097956795379517951794E118F10A430B1B
:10283000560BC90BD00998F023957E9173957A3386
:1028400008F070E37C932013B8F77E9170617D935C
:1028500030F0839571E37D9370E32A95E1F71124BD
:10286000EF90FF900F911F91CF91DF91992787FDF6
:0828700090950895F894FFCF44
:102878000A0002000E00007A44050100000005006D
:1028880000000A0000001900000032000000640087
:102898000000E8030000881300001027000050C360
:1028A8000000A0860100D084000020AA44007F8D8B
:1028B8005B000300000001000000FF0000000100B1
:1028C800000001000000E8030000E8030000111008
:1028D8000F860C860C535445503A006B487A004DCD
:1028E800487A00465245513A004F4E0053415645EA
:1028F8004420544F20454550524F4D00202000564B
:10290800455253494F4E3A345F3100000000008071
:042918000CB50E00EC
:00000001FF
